:1000000012C02BC02AC029C028C027C026C025C0C6
:1000100024C023C022C06CC020C01FC01EC01DC091
:100020001CC01BC01AC011241FBECFE5D4E0DEBF28
:10003000CDBF10E0A0E6B0E0E8EDF1E002C0059031
:100040000D92A036B107D9F710E0A0E6B0E001C0EC
:100050001D92A136B107E1F739C0D2CF40E050E0A0
:100060004817590768F420E030E0275E3F4F60E70B
:100070002E343607D0F34F5F5F4F4817590798F378
:10008000089587B38F6387BB88B3807F806388BB05
:1000900084B3837C836084BB85B3807C85BB81B360
:1000A00086EF81BB82B382E382BB08958BB18C7FE4
:1000B00080648BB98AB1827980698AB986E880BD0B
:1000C00080B5807780BD8FEC89B90895CFE5D4E005
:1000D000DEBFCDBF10926000D4DF8FB78F778FBFA8
:1000E000E5DF8FB780688FBF88B3866088BBFFCF9E
:1000F0001F920F920FB60F9211242F933F934F939D
:100100005F936F937F938F939F93AF93BF93EF937F
:10011000FF938CB1282F33272B31310521F02B355C
:10012000310531F00EC081E080936000C09A43C079
:10013000929A809160008130F1F582E080936000B6
:100140003AC080916000823091F52234310591F0FF
:100150002334310524F42134310541F028C02334FF
:10016000310561F02434310589F021C082B38F7EDE
:1001700080620FC082B38F7D806103C082B38F7EA7
:10018000806282BB88B38F7D806107C082B38F7D20
:10019000806182BB88B38F7E806288BB84E690E0FA
:1001A0005DDF82B3806382BB88B3806388BB1092BB
:1001B0006000C0989298FF91EF91BF91AF919F918D
:1001C0008F917F916F915F914F913F912F910F9000
:0801D0000FBE0F901F9018955F
:00000001FF
